:020000040800F2
:10000000700E0024390300083D100090970F0090F7
:10001000450300087B030090D71C009000000000FF
:1000200000000000000000000000000041100090EF
:100030007D030090000000003F10009043100090EE
:100040005303000853030008530300085303000838
:100050005303000853030008530300085303000828
:100060005303000853030008530300085303000818
:100070005303000853030008530300085303000808
:1000800053030008530300085303000853030008F8
:1000900053030008530300085303000853030008E8
:1000A00053030008530300085303000853030008D8
:1000B000530300084910009053030008530300083D
:1000C00053030008530300085303000853030008B8
:1000D00053030008111300085303000853030008DA
:1000E00053030008530300080000000053030008F6
:1000F0005303000853030008530300085303000888
:100100005303000853030008E51000905303000850
:100110005303000853030008530300085303000867
:100120005303000853030008530300085303000857
:100130005303000853030008530300085303000847
:1001400000000000000000000000000000000000AF
:100150005303000853030008530300085303000827
:100160005303000853030008530300085303000817
:100170005303000853030008530300085303000807
:1001800053030008530300085303000853030008F7
:1001900053030008530300085303000853030008E7
:1001A00053030008530300085303000853030008D7
:1001B00053030008530300085303000853030008C7
:1001C00053030008530300085303000853030008B7
:1001D00053030008530300085303000853030008A7
:1001E0005303000853030008530300085303000897
:1001F0005303000853030008530300085303000887
:100200005303000853030008530300085303000876
:100210005303000853030008530300085303000866
:1002200053030008530300085303000800000000B4
:1002300053030008530300080000000053030008A4
:100240005303000853030008530300085303000836
:100250005303000853030008530300085303000826
:100260005303000853030008530300085303000816
:100270005303000853030008530300080000000064
:1002800053030008000000005303000800000000B2
:10029000000000005303000800F002F800F03CF8F2
:1002A0000AA090E8000C82448344AAF10107DA45D1
:1002B00001D100F031F8AFF2090EBAE80F0013F0E7
:1002C000010F18BFFB1A43F0010318472812000062
:1002D00048120000103A24BF78C878C1FAD85207F3
:1002E00024BF30C830C144BF04680C6070470000B0
:1002F0000023002400250026103A28BF78C1FBD82F
:10030000520728BF30C148BF0B6070471FB501F0CE
:10031000E3F81FBD10B510BD00F0AAF81146FFF7B5
:10032000F5FF01F065F800F0C8F803B4FFF7F2FF3D
:1003300003BC01F01FF80000094880470948004746
:10034000FEE7FEE7FEE7FEE7FEE7FEE7FEE7FEE785
:10035000FEE7FEE704480549054A064B70470000E2
:100360008D1200089902000870020024700E00240B
:100370007004002470040024704753EA020C00F05B
:1003800069802DE9F04B4FF00006002B1FBFB3FA38
:1003900083F503FA05F424FA05F65E4012BF16430E
:1003A000B2FA82F502FA05F4C5F120051EBF22FA61
:1003B00005FC44EA0C04203556EA044C4FEA144488
:1003C00018BF641C4FF000084FF00009904271EB19
:1003D000030C39D3002919BFB1FA81F701FA07F6E6
:1003E000B0FA80F700FA07F6C7F120071EBF20FA1F
:1003F00007FC46EA0C062037B6FBF4FCA7EB050722
:10040000103F07F01F0BCBF120060CFA0BFB2CFA68
:1004100006F644BFB3460026202FA4BF5E464FF029
:10042000000B5BEA060C08BF4FF0010B19EB0B0940
:10043000ABFB027C48EB0608C01B06FB02CC0BFBA7
:1004400003CC71EB0C01C1E70B460246414648461E
:10045000BDE8F08B13B54FF000004FF00001AFF393
:100460000080BDE81C407047704770477047704778
:10047000754600F02BF8AE4605006946534620F05D
:100480000700854618B020B5FFF764FFBDE820409F
:100490004FF000064FF000074FF000084FF0000B40
:1004A00021F00701AC46ACE8C009ACE8C009ACE8F3
:1004B000C009ACE8C0098D46704710B50446AFF3DB
:1004C00000802046BDE81040FFF72FBF004870476E
:1004D0000C02002440F2154CC9F2000C604740F6B3
:1004E000055CC9F2000C604740F6F74CC9F2000CFD
:1004F000604740F6EF6CC9F2000C604740F6F97CAB
:10050000C9F2000C604740F6997CC9F2000C6047C4
:1005100041F2550CC9F2000C604741F29D0CC9F242
:10052000000C604741F2C91CC9F2000C604741F25F
:10053000CD4CC9F2000C604740F2150CC9F2000C1A
:10054000604740F6856CC9F2000C6047F0B5BFF318
:100550004F8FBFF36F8F1D4900200860BFF34F8F8F
:10056000BFF36F8F1A4C216841F400312160BFF353
:100570004F8FBFF36F8F164970310860BFF34F8FF5
:10058000081F006843F6FF75104E1036C0F34E3159
:10059000C0F3C90305EA4112184642EA8077376082
:1005A000401EFAD2491EF5D2BFF34F8F206840F4A7
:1005B00080302060BFF34F8FBFF36F8F03484C3004
:1005C000016841F004010160F0BD000050EF00E05F
:1005D00014ED00E00248016841F00101016070473C
:1005E000200400582DE9F84F6C4C00224FF0B04A1F
:1005F0004FF0010B4FF0030E4FF00F090B680BFA91
:1006000002F73B40BB4270D14D68022D01D0122D44
:1006100012D1D50800EB850CDCF820605507ED0EF3
:1006200009FA05F826EA0806D1F8108008FA05F854
:1006300048EA0608CCF82080D0F80080560091F8EF
:1006400004C00EFA06F50CF0030C28EA05080CFAB3
:1006500006FC4CEA080CC0F800C0D1F804C0BCF19C
:10066000010F08D0BCF1020F05D0BCF1110F02D070
:10067000BCF1120F16D1D0F808C0D1F80C802CEACA
:10068000050C08FA06F848EA0C08C0F80880D0F80B
:1006900004C02CEA070C0F79C7F30017974047EA0C
:1006A0000C074760C768AF438D68B5403D43C560E0
:1006B0004D68ED006BD53A4D2E6846F002062E606F
:1006C0002D6822F0030606F1B04605F002050095FC
:1006D000D6F808C495072F0F09FA07F52CEA050C80
:1006E000304DA84202D100252EE050E02E4DA84208
:1006F00001D1012528E02D4DA84201D1022523E09A
:100700002B4DA84201D103251EE02A4DA84201D15C
:10071000042519E0284DA84201D1052514E0274DF4
:10072000A84201D106250FE0254DA84201D1072599
:100730000AE0244DA84201D1082505E0224DA84237
:1007400001D1092500E00A25BD4045EA0C05C6F89F
:10075000085425684E689D43F60300D51D43256067
:1007600065684E689D43B60300D51D436560DAF8A1
:10077000005056464F689D43FF0200D51D4335602B
:1007800075684F689D43BF0200D51D437560521CBC
:10079000102AFFF433AFBDE8F88F00008000005846
:1007A000F44402580000025800040258000802589D
:1007B000000C025800100258001402580018025889
:1007C000001C025800200258002402580AB101837C
:1007D00070474183704700000148806870470000FF
:1007E0001400002402488168027811448160704737
:1007F00014000024032010B500F058F80F2000F07A
:1008000007F808B1012010BD00F022F8002010BD4B
:1008100070B50D4D04464FF47A712878B1FBF0F0B5
:100820000A490968B1FBF0F000F05AFC48B9102CF5
:1008300007D200222146501E00F018F800206C60FC
:1008400070BD012070BD00001400002400000024D1
:100850007047002809DB012100F01F029140400988
:10086000800000F1E020C0F8001170470E4BF0B49A
:100870001B68C3F30223C3F10704042C00D904242A
:100880001D1D072D01D2002300E0DB1E012606FA04
:1008900004F56D1E0D409D409E40761E164045EAB3
:1008A0000601F0BC00F056BD0CED00E0064A00F079
:1008B000070110684FF6FF03184040EA0120034982
:1008C00008431060704700000CED00E00000FA05DE
:1008D0002DE9F047DFF8BC9104460E46D9F8000038
:1008E00000F00700B0420CD2D9F8001021F0070147
:1008F0003143C9F80010D9F8000000F00700B042F9
:100900007ED12078DFF89081800707D5D8F80010D5
:10091000E26821F00F011143C8F800102078C007E9
:1009200062D0D8F80010A26821F470611143C8F8B1
:10093000001059496068183902281CD003281DD0BE
:10094000096801281DD04907002960DA524F083F85
:10095000396821F0070101433960FFF73DFF054683
:10096000606841F28831022813D003281ED0012884
:100970008A4627D034E009688903E5E709688901D8
:10098000E2E7C905E0E7FFF727FF411B514501D921
:1009900023E08A463868C0F3C2000228F3D123E07E
:1009A000FFF71AFF411B514501D916E08A46386806
:1009B000C0F3C2000328F3D116E0FFF70DFF411B7F
:1009C00051450AD83868C0F3C2000128F5D10BE0C0
:1009D000FFF702FF411B514502D90320BDE8F08714
:1009E000386810F0380FF3D1D9F80010484601F0FC
:1009F0000701B1420DD9016821F00701314300E040
:100A000005E00160006800F00700B04201D001205D
:100A1000E4E72078400707D5D8F80010226921F0D4
:100A200070011143C8F80010207801071B4805D554
:100A30000168626921F07001114301602178C906E3
:100A400005D50168A26921F4E061114301602078B5
:100A5000800607D51149091D0868E26920F0700079
:100A60001043086000F066F8D8F800104FF4807268
:100A700092FAA2F201F47061B2FA82F2D140084A0D
:100A8000515CC840074908600F20FFF7C1FE0020F5
:100A9000A4E7000000200052184402581C440258E9
:100AA000E21400080000002410B5FFF713FD084908
:100AB0000968012292FAA2F201F00F01B2FA82F261
:100AC000D140044A515CC8400349086010BD000091
:100AD00018440258E21400080400002410B5FFF77F
:100AE000E3FF07490968102292FAA2F201F07001AF
:100AF000B2FA82F2D140034A515CC84010BD0000F6
:100B00001C440258E214000810B5FFF7CDFF074956
:100B100009684FF4807292FAA2F201F4E061B2FA2D
:100B200082F2D140024A515CC84010BD1C440258B8
:100B3000E21400083548F0B50068364D10F0380171
:100B4000334809D00411082904D0334E10290BD0A2
:100B500018290BD02046F0BD29688906FBD52968E5
:100B6000C1F3C101C840F0BD3046F0BD274918317E
:100B70000A68096812F00302284BC1F305111B68CB
:100B8000274F03F001033F68DFED260AB7EE001A96
:100B9000C7F3CC0717FB03F300EE103A224BB8EE75
:100BA000400A06D0012A01D0022A2BD0B4FBF1F072
:100BB00008E02A68920603D52A68C2F3C102D04031
:100BC000B0FBF1F001EE900A1868B8EE612AC0F3AC
:100BD000080001EE900A1868F8EE611A40EE201A3B
:100BE00031EE810A22EE000AC0F34620401C00EEDE
:100BF000900AF8EE600A80EE201ABCEEC10A10EEF0
:100C0000100AF0BDB6FBF1F0DCE70000104402581A
:100C10000090D0030044025840787D012C440258D3
:100C20003444025800000039304402582DE9F05F86
:100C300004460078DFF8FC8341F28839DFF8F8A336
:100C4000FE4DC0074ED0D8F800104046C1F3C20197
:100C500002291AD00068C0F3C200032805D1DAF8CF
:100C6000000000F0030002280FD06068B0F5803F5C
:100C700012D010B1B0F5A02F19D0286820F4803020
:100C80002860286820F4802009E02868800329D59E
:100C90006068002874D025E0286840F4803028601F
:100CA000606890B1FFF798FD06464F4609E0286856
:100CB00040F480202860EFE7FFF78EFD801BB842EC
:100CC0007DD828688003F7D50CE0FFF785FD064640
:100CD0004F4604E0FFF780FD801BB842F0D828683B
:100CE0008003F7D42078D64F80075AD5D8F8001063
:100CF00040464FF47C3B11F0380F13D00068C0F32E
:100D0000C200032803D1DAF8000080070AD0E068A7
:100D1000A8B3296821F0190101432960FFF75CFDA0
:100D200006461DE02868400702D5E0680028B1D0DB
:100D30002868E16820F0190008432860FFF74CFD9F
:100D4000064604E0FFF748FD801B0228B8D8286853
:100D50004007F7D507E0FFF73FFD801B0228AFD81B
:100D600028684007F7D538689BFAABF220F47C314D
:100D70002069B2FA82F290400143396011E000E04C
:100D8000AEE0286820F001002860FFF725FD064648
:100D900004E0FFF721FD801B022891D82868400756
:100DA000F7D42078C00655D5D8F8001040464FF04B
:100DB000F84BC1F3C201012917D0006800E0EDE053
:100DC000C0F3C200032805D1DAF8000000F00300E8
:100DD00001280AD0E069002828682CD040F0800063
:100DE0002860FFF7F9FC064616E02868C00502D522
:100DF000E069802874D138689BFAABF220F0F841A2
:100E0000206AB2FA82F290400143396022E0FFF793
:100E1000E3FC801B022899D82868C005F7D53868FC
:100E20009BFAABF2216AB2FA82F220F0F8409140CC
:100E3000084338600EE020F080002860FFF7CCFC0B
:100E4000064604E0FFF7C8FC801B022887D8286804
:100E5000C005F7D42078000724D5774F60694C3758
:100E6000002838680FD040F001003860FFF7B4FC6C
:100E7000064604E0FFF7B0FC801B02288DD83868D6
:100E80008007F7D50EE020F001003860FFF7A4FCE2
:100E9000064604E0FFF7A0FC801B02287ED83868D5
:100EA0008007F7D42078800623D5A0690028286819
:100EB0000FD040F480502860FFF78EFC064604E017
:100EC000FFF78AFC801B022868D828688004F7D5C1
:100ED0000FE020F480502860FFF77EFC064605E016
:100EE000D6E0FFF779FC801B022857D828688004D9
:100EF000F7D42078400744D5524F386840F48070CA
:100F00003860FFF769FC064604E0FFF765FC801BCC
:100F1000642843D83868C005F7D5474FA0684837DC
:100F200001280AD008B1052811D0386820F0010046
:100F30003860386820F0040002E0386840F00100B2
:100F40003860A06888B1FFF747FC064609E03868BA
:100F500040F004003860F0E7FFF73EFC811B494594
:100F60001CD838688007F7D50BE0FFF735FC06463C
:100F700004E0FFF731FC811B49450FD83868800732
:100F8000F7D4606AF0B3D8F80010C1F3C2010329A6
:100F90007ED00228286820F0807000E079E0286088
:100FA00003D0FFF719FC044687E0FFF715FC06465F
:100FB00004E0FFF711FC801B02287BD82868800121
:100FC000F7D4DAF8001040F2F3329143E26A41EAD2
:100FD0000211A26A1143CAF8001094F834004FF4C9
:100FE000FE02218E4002491EA0F5007080B2C1F3BE
:100FF00008010843218F491E02EA0141084394F881
:101000003C1000E05CE0491E120202EA0161084364
:101010000949083108600B1D19684FF6F872A06C79
:10102000914392FAA2F2B2FA82F29040014319601F
:10103000014809E01044025828440258004402586C
:101040000444025800480258001D0168226C21F037
:101050000C01114301600168626C21F0020111432F
:101060000160016841F480310160016841F40031A0
:101070000160016841F480210160016841F00101D3
:101080000160286840F080702860FFF7A5FB01E050
:1010900018E00FE0044604E0FFF79EFB001B022867
:1010A00008D828688001F7D50AE0FFF795FB001BF8
:1010B000022802D90320BDE8F09F28688001F4D4FB
:1010C0000020F8E70120F6E74FF0E0210428086946
:1010D00003D020F004000861704740F00400FAE7F4
:1010E000401EB0F1807F10B501D3012010BD4FF03C
:1010F000E02460610F21601700F02CF90020A0614E
:1011000007202061002010BD10B5006886B01B4983
:10111000884230D11A48016841F00101016000683D
:1011200000F00100059016481030016841F01001F0
:10113000016000680121134C00F0100005904FF48D
:10114000007000900220CDE901010390072069465C
:1011500004902046FFF746FA4FF480612046009144
:101160006946FFF73FFA2520FFF773FB032225208E
:101170001146FFF77BFB06B010BD000000100140D8
:10118000E04402580000025830B500681149884216
:101190000CD1114A5088010408D411464FF00003C5
:1011A0004404097806D50A2901D0538030BD40F4A3
:1011B00000400DE00D2909D0084DC0F30D04401C7E
:1011C00080B2C72829555080EFD830BD40F4804008
:1011D000508030BD001001400C0000242800002485
:1011E00070B5284C9CB0256825F004052560254C79
:1011F00000260C34256845F440452560256805F433
:1012000040451B952568AD04FCD5012400940CAD28
:1012100003962404019402240994CDE90A41079617
:10122000082485E80D00CDE910466846FFF7FEFC6E
:1012300088B93F2013900320CDE914064020010116
:10124000CDE91640CDE9180150201A90022113A8CB
:10125000FFF73EFB10B101201CB070BD0A480168C9
:1012600041F0800101600848F430016841F002015A
:101270000160006800F002001B90FFF7ABF900204E
:10128000EAE700000C480258004402581C48016874
:1012900041F4700101601B49086840F001000860DA
:1012A000184A0020103210600A68174B1A400A6072
:1012B000144A18321060121D1060121D1060114A7D
:1012C00028321060121D1060121D1060121D106077
:1012D000121D1060121D1060121D1060121D106092
:1012E0000A6822F480220A60064960310860012001
:1012F0000649C1F80801C0060149803908607047F5
:1013000088ED00E0004402587FEDF6EA00800051CD
:1013100070B50D4D00240D48FFF7E1F802E0641CA4
:10132000AC4204D80948FFF7DFF82028F7D10024A1
:1013300002E0641CAC4206D8054901220348FFF7CD
:10134000D8F80028F5D170BDFFFF0100F00000249F
:101350000C0000240907090E002804DB00F1E0203E
:1013600080F80014704700F00F0000F1E02080F8D2
:10137000141D70477047000010B504460420FFF7A5
:10138000A3FE0148046010BD0800002470B50024CD
:1013900005464FF47A7603E0304600F005F8641C09
:1013A000AC42F9D370BD000070B54FF0E0250021CC
:1013B0006C69094AAB6912685043AA699A42FCD029
:1013C00002D2A3EB020302E0A4EB02063344194469
:1013D00013468142F1D370BD080000240349CA6955
:1013E0005206FCD5C2B20A857047000000100140C9
:1013F000FFF7ACF8FFF7FEF9042302220521A02035
:10140000FFF7EEFE4FF4C870FFF7B6FF4FF4E13080
:1014100000F046F8FFF772F8FFF775F8C72140F2C1
:10142000F310FFF775F8C7214FF0FF30FFF775F89D
:10143000154D0024154E4FF496780A20FFF7A6FFAD
:10144000FFF770F8401CFFF772F8FFF76BF84045A4
:1014500002D10020FFF76BF828780106EDD500F0E7
:101460003F014FF0FF320027CB0FA1FB020C03FB23
:1014700002C201FB072331684218634104A0FFF751
:101480005BF82C70D9E70000200000242400002421
:10149000484947483A256C6C642075730D0A000072
:1014A0000B490A4A10B5C1E9002000208860C860D5
:1014B000086188610C2048610846FFF742F8BDE8E2
:1014C0001040044901220248FFF713B80010014000
:1014D000F00000240C0000244FF04070E1EE100AF0
:1014E0007047000000000102030401020304060724
:1014F000080900001415000800000024280000005E
:10150000D40200083C15000828000024480E000002
:10151000F00200080090D0030090D003000000000B
:1015200000000000000000000100000010000000AA
:0C153000000000000000000000000000AF
:0200000490006A
:1000000003681B0A28BF41F08001E42900F00E803C
:10001000002070470FB4044910B503AA029800F0FD
:100020003DF910BC5DF814FB100000242DE9F041EF
:100030008046D21D22F007020025D2E90002F529F0
:1000400015A614D0011E72F1000106DA0023D0EBD0
:10005000030063EB020211A608E0D8F800108B073A
:1000600001D50FA602E0490701D50EA601251146CC
:10007000002408F1240704E000F072F830323A5509
:10008000641C50EA0102F7D12B4632462146404615
:10009000BDE8F04100F0A9B8000000002D0000000C
:1000A0002B000000200000002DE9F0410F4605461E
:1000B000002028622846E968884770B3252805D0C3
:1000C000D5E901219047286A401CF2E7E9682846F3
:1000D000002688476C2804460AD0682C08D04C2C8F
:1000E00035D06A2C31D0742C31D07A2C2FD016E038
:1000F000E968064628468847B042044608D16C2E77
:1001000023D04FF480662846E9688847044606E015
:100110006C2E03D04FF4807601E01EE04026E4B15F
:10012000A4F14100192802D8203446F400663A466A
:10013000214628462E60FFF763FF60B1012808D0F2
:10014000FF1D27F007070837B4E78026DBE7002606
:10015000D9E73F1DAEE72046B2E7286ABDE8F08147
:1001600030B5B0F10A024FEA900E71F100034EEA89
:10017000817EB0EB0E0061EB91014FEA101E4EEA5A
:10018000017E10EB0E0041EB11114FEA102E4EEAEA
:10019000016E10EB0E0041EB11214FEA104E4EEABA
:1001A000014E10EB0E0041EB1141401841F10001EE
:1001B0004FEAD00040EA41704FEAD10110EB8005D0
:1001C0004FEA810444EA907444EB01046D1944EB56
:1001D0000404521BA3414FF0000348BF0A3200D56C
:1001E00030BD401C41F1000130BD2DE9F0470D4606
:1001F00099469246044600F124080168880604D511
:10020000E06921F01001216000E00120A84201DD39
:10021000471B00E00027A1697A1902EB0900081AC0
:10022000A0612078C00602D42046AFF300800026EB
:1002300008E0D4E901211AF806009047206A401C22
:10024000761C20624E45F4DB2078C0060AD5204695
:10025000AFF3008006E0D4E9012130209047206A06
:10026000401C2062381EA7F10107F4DC07E0D4E946
:10027000012118F805009047206A401C2062281EC2
:10028000A5F10105F3DC2046AFF3008020780006DD
:1002900002D50220BDE8F0870120FBE7074B70B5CF
:1002A0000D467B4400F011F80446284600F020F883
:1002B00010B14FF0FF3070BD204670BD371100788F
:1002C00001694A1C02610878704700B58FB0CDE91A
:1002D00001310021059105497944CDE9031011460A
:1002E0006846FFF7E1FE0FB000BD0000E5FFFFFF2D
:1002F000007B00F08000704740F6353CC0F6000CF3
:10030000604740F6A92CC0F6000C604740F2E55C5F
:10031000C0F6000C604740F66D0CC0F6000C60475C
:1003200040F6530CC0F6000C604741F2091CC0F6C1
:10033000000C604740F2CD7CC0F6000C604740F2F4
:10034000E57CC0F6000C604740F2D97CC0F6000C9A
:10035000604741F2891CC0F6000C604740F27B3CCC
:10036000C0F6000C604740F6DD2CC0F6000C60477C
:1003700040F6093CC0F6000C6047FEE770470000FD
:1003800010B528B190F83510022903D080214165BD
:10039000012010BD1D4A4FF4956301688C189C42E2
:1003A00007D8042280F83520086820F00100086092
:1003B00029E00C6824F00E040C6001680A440A6805
:1003C00022F001020A60016E0A6822F480720A605B
:1003D00090F85C30012202FA03F10D4B1960D0E96C
:1003E00019134B60C16E31B10B6823F480730B603D
:1003F000D0E91C134B60002180F8341080F83520C0
:10040000016D01B18847002010BD0000F0FFFDBF65
:100410000454025810B5FFF76FFF084909684FF4FC
:10042000807292FAA2F201F47061B2FA82F2D140C3
:10043000034A515CC8400349086010BD1844025883
:10044000E21400080000002410B5FFF75AFF074926
:100450000968102292FAA2F201F07001B2FA82F257
:10046000D140034A515CC84010BD000020440258EE
:10047000E2140008364930B50A68096812F0030230
:10048000344BC1F305311B68334C03F0100324686F
:10049000DFED320AB7EE001AC4F3CC0414FB03F309
:1004A00000EE103A2E4BB8EE400A07D02D4C012A30
:1004B00001D0022A4AD0B4FBF1F10BE0244C283CD5
:1004C00022689506284A03D52468C4F3C104E24093
:1004D000B2FBF1F101EE901A1968B8EE612AC1F38E
:1004E000080101EE901A1968F8EE611A40EE201A20
:1004F00031EE810A22EE000AC1F34621491C00EECA
:10050000901AF8EE600A80EE201AFCEEC10AC0EDE7
:10051000000A1968C1F30641491C00EE901AF8EE72
:10052000600A80EE201AFCEEC10AC0ED010A1968CB
:10053000C1F30661491C00EE901AF8EE600A80EEE5
:10054000201ABCEEC10A80ED020A30BD074ABFE79F
:10055000284402582C4402583C44025800000039F8
:100560003844025800093D000090D00340787D01D6
:10057000364930B50A68096812F00302344BC1F3FA
:1005800005511B68334C03F480732468DFED320A95
:10059000B7EE001AC4F3CC0414FB03F300EE103AD8
:1005A0002E4BB8EE400A07D02D4C012A01D0022A6A
:1005B0004AD0B4FBF1F10BE0244C283C22689506AC
:1005C000284A03D52468C4F3C104E240B2FBF1F128
:1005D00001EE901A1968B8EE612AC1F3080101EE24
:1005E000901A1968F8EE611A40EE201A31EE810A6D
:1005F00022EE000AC1F34621491C00EE901AF8EEE3
:10060000600A80EE201AFCEEC10AC0ED000A1968EB
:10061000C1F30641491C00EE901AF8EE600A80EE24
:10062000201AFCEEC10AC0ED010A1968C1F3066187
:10063000491C00EE901AF8EE600A80EE201ABCEE1B
:10064000C10A80ED020A30BD074ABFE728440258BC
:100650002C440258444402580000003940440258D7
:1006600000093D000090D00340787D01704770473D
:1006700070B51E4E3078010613D41D4C41064FF65E
:10068000F5750FD540F0800030700021204600F055
:100690000DFB70602068016A294001622068016AD0
:1006A000016270BD00217160402030702068026AD4
:1006B00041F211131A4207D1026A9B101A4203D168
:1006C000028822F001020280206841622068016AEB
:1006D000294001622068016A41F00201016220683C
:1006E000018841F00101018070BD0000200000245C
:1006F000CC0100242DE9F041044690F83C000D4661
:1007000001283CD0012684F83C60022084F83D009A
:10071000A2B3042A45D02068082A54D0D5E900277E
:10072000E968036A23F480530362D0F81CC0036AAB
:100730002CF4407C4CEA07274FF6FF7C27F47047E7
:100740000CEA01313943C1614FF4204723F42043BF
:1007500007EA02321A4302622068C16921F440614B
:10076000C1612068C169AA6841EA0221C16184F8B7
:100770003D60002084F83C00BDE8F08101E00220EB
:10078000FAE7EB682068D5E9001200F0A5FE2068C2
:10079000816921F00C01816120688169AA68114397
:1007A0000FE0EB682068D5E9001200F0D5FE206864
:1007B000816921F44061816120688169AA6841EA08
:1007C00002218161D3E7D5E9002C2F7B016A21F456
:1007D00080710162C169036A21F0030141EA0C01E1
:1007E00021F0F00C39074FF4206723F4206307EA67
:1007F00002221A434CEA1161C16102622068C16998
:1008000021F00C01C1612068C169AA681143ADE7FC
:1008100010B5040003D094F83D0010B107E00120AA
:1008200010BD002084F83C00204600F00DF80220A6
:1008300084F83D002068211D00F05AFC012084F856
:100840003D00002010BD0000154800B587B00168CC
:1008500041F008010160006800F0080005901048B0
:100860000838016841F0010101600068032100F0CF
:10087000010005900120009002200190CDE90201C5
:10088000049069460748FFF741FD0022022132200B
:10089000FFF741FD3220FFF743FD07B000BD000028
:1008A000E84402580000025810B50268044631B10D
:1008B000042908D0082915D00C2908D116E0D068E1
:1008C00040F0020002E0D06840F00400D0602068F0
:1008D000012200F06DFC2068018841F001010180D7
:1008E000002010BDD06840F00800EFE7D06840F06D
:1008F0001000EBE770B50446006801694FF0000591
:10090000C943890715D4C168C943890711D4E91EB1
:10091000016101202077206880698007204602D08D
:10092000FFF7A6FE04E000F0A5F8204600F07AF9F3
:10093000257720680169C943490717D4C168C943AD
:10094000490713D46FF00401016102202077206869
:10095000806910F4407F204602D0FFF789FE04E052
:1009600000F088F8204600F05DF9257720680169DD
:10097000C943090716D4C168C943090712D46FF0E7
:1009800008010161042020772068C06980072046A3
:1009900002D0FFF76DFE04E000F06CF8204600F096
:1009A00041F9257720680169C943C90617D4C16890
:1009B000C943C90613D46FF01001016108202077E4
:1009C0002068C06910F4407F204602D0FFF750FE37
:1009D00004E000F04FF8204600F024F92577206865
:1009E0000169C943C90708D1C168C943C90704D10E
:1009F000891E0161204600F043F9206801696FF00B
:100A00008005C943090607D4C168C943090603D450
:100A100005612046FFF72AFE20680169C943C90520
:100A200007D4C168C943090603D405612046FFF70E
:100A30001DFE20680169C943490609D4C168C9433C
:100A4000490605D46FF040010161204600F050F9DD
:100A500020680169C94389060BD4C168C943890666
:100A600007D46FF0200101612046BDE87040FFF718
:100A7000FEBD70BD704770B5044690F83C000D4651
:100A800001280ED0012684F83C60022084F83D0045
:100A90000C2A45D007DC5AB1042A1BD0082A78D189
:100AA0002CE0022070BD102A4ED0142A71D15DE0D6
:100AB000206800F08FFB2068816941F008018161A6
:100AC0002068816921F004018161206881692A69B7
:100AD000114311E0206800F0CBFB2068816941F4EC
:100AE000006181612068816921F4806181612068F1
:100AF00081692A6941EA022181614AE0206800F0A7
:100B0000FFFB2068C16941F00801C1612068C1692B
:100B100021F00401C1612068C1692A69114311E013
:100B2000206800F031FC2068C16941F40061C161B6
:100B30002068C16921F48061C1612068C1692A69A6
:100B400041EA0221C16124E0206800F053FC2068E2
:100B5000416D41F0080141652068416D21F00401BB
:100B600041652068416D2A69114311E0206800F059
:100B700077FC2068416D41F4006141652068416D5A
:100B800021F4806141652068416D2A6941EA0221B2
:100B9000416584F83D60002084F83C0070BD10B5CC
:100BA000040003D094F83D0010B107E0012010BD0F
:100BB000002084F83C00204600F00CF8022084F865
:100BC0003D002068211D00F093FA012084F83D00CB
:100BD000002010BD114800B587B0016841F0020146
:100BE0000160006800F0020005900C4808380168B8
:100BF00041F0020101600068012100F0020005904F
:100C000002200090CDE901010321CDE90310044841
:100C10006946FFF77BFB07B000BD0000E8440258BF
:100C2000000402587047000010B501220446006815
:100C300000F0BEFA0D48216881420BD00C48814279
:100C400008D00C48814205D00B48814202D00B48A5
:100C5000814203D1486C40F4004048642068018818
:100C600041F001010180002010BD000000000140A2
:100C700000040140004001400044014000480140A0
:100C800009490878020606D4420604D5C2439206F2
:100C900002D0401C0870704740F0800008704FF090
:100CA000FF304860704700002000002490F83C307E
:100CB0000022012B0AD0012380F83C3041B10429E5
:100CC00009D008290AD00C290DD10AE0022070476A
:100CD00001684A6B07E001688A6B04E00168CA6B2F
:100CE00001E001680A6C002180F83C101046704752
:100CF00070477047704790F8791090F87A00084371
:100D00007047000070B502680446D06913689168A6
:100D100010F00F0F64D0594D03F490760D40354319
:100D200076D0C50707D0DD0505D501251562E26F30
:100D300042F00102E267820708D5CA0706D025689B
:100D400002222A62E26F42F00402E267420708D5FB
:100D5000CA0706D0256804222A62E26F42F0020226
:100D6000E26702070ED503F0200201F080552A4306
:100D700052EAC17206D0256808222A62E26F42F068
:100D80000802E267E26F002A3AD0800608D503F035
:100D9000200001F08051084302D0204600F0A1FC61
:100DA000E06F000703D42068806840062AD52046FB
:100DB00000F089FC2068816849061ED5816821F011
:100DC00040018160606FC0B12D490165606FFFF720
:100DD000D7FA002814D0606F016DBDE87040084755
:100DE000850615D503F0200501F0805635430FD058
:100DF0002046BDE8704000F074BC2046FFF77AFF43
:100E000070BD05E02046FFF775FF0020E067F7E7BB
:100E1000C6024FF020050CD54E020AD5E803106239
:100E200084F8795084F87A502046BDE87040FFF786
:100E300060BF06060AD503F0800601F400010E43E8
:100E400004D02046BDE8704000F0DABE41060BD564
:100E5000590609D51168204621F04001116084F837
:100E6000795000F097F8CBE70002C9D55800C7D5F4
:100E7000106820F080401060C2E700000100001000
:100E8000B316009010B5040003D094F8790010B1A7
:100E900007E0012010BD002084F878002046FFF70D
:100EA00044FA242084F879002068016821F00101C7
:100EB0000160204600F050FC0128EBD0606B10B1BF
:100EC000204600F064FB2068416821F490414160B5
:100ED0002068816821F02A0181602068016841F062
:100EE000010101602046BDE8104000F0B4BB90F85D
:100EF0007A30202B4CD1B9B1B2B190F87830012BB7
:100F000046D0012380F878304166A0F86820A0F828
:100F10006A20FF228168B1F5805F07D07F2351B13D
:100F2000B1F1805F0CD010E001207047016921B958
:100F300040F2FF1107E0016909BBA0F86C2004E052
:100F40000169E1B13F21A0F86C100021C1672222A4
:100F500080F87A2080F8781001688A6842F00102EF
:100F60008A6001680A6892000CD50A6842F48072AF
:100F70000A600068816841F08051816006E0A0F855
:100F80006C30E2E7086840F4907008600020704719
:100F9000022070477047FEE7144870B586B00168BC
:100FA00041F004010160016801F00401059101684C
:100FB00041F010010160006800260325694600F039
:100FC0001000059008200124CDE900060848CDE96D
:100FD0000245FFF79BF920206946CDE90006054848
:100FE000CDE90245FFF792F906B070BDE044025822
:100FF00000100258000802580E4810B586B001686B
:1010000041F001010160006869460B4C00F00100ED
:10101000059002200090012001900290032003908F
:101020002046FFF773F9012220460221FFF782F9DB
:1010300006B010BDE04402580000025870477047E7
:101040007047FFF77CB900000148FFF753BC000070
:1010500070010024104A10B504460E48C2E9000190
:101060000020C2E9020410611046FFF798FD0A490A
:1010700060200C22403108606008486002208860CF
:101080000548FFF7F8FCBDE8104003480C21FFF7C6
:10109000CBBD000000040040700100247FB5104C5F
:1010A00000250E4AC4E9025025612046C4E900210A
:1010B000FFF7AEFB01206946002202950395CDE9BA
:1010C00000502046FFF716FB00212046FFF7ECFBFF
:1010D0002068C16841F00101C1607FBD000C004083
:1010E000CC0100240148FFF705BC0000CC0100241E
:1010F0002DE9F04702884FF0804A254C254D264EB9
:10110000A042264F264B09D0504507D0A84205D013
:10111000B04203D0B84201D0984204D122F0700C02
:101120004A6842EA0C02DFF87CC0DFF87C80A0420B
:10113000DFF878900FD050450DD0A8420BD0B042C8
:1011400009D0B84207D0984205D0604503D0404549
:1011500001D0484503D122F44075CA682A438D8ADC
:1011600022F080022A4302808A68C2620A880285CD
:10117000A04207D0984205D0604503D0404501D039
:10118000484501D1098A018601214161BDE8F08706
:10119000000001400004004000080040000C004036
:1011A000000401400040014000440140004801406B
:1011B000012310B5046A8B409C430462036A8A4091
:1011C0001343036210BD000001480C21FFF76EBD00
:1011D000700100242DE9F043026A22F0010202624C
:1011E000056A4268836925F002051B4C1C4E2340AA
:1011F0000C6823F003031B4F1C438B68DFF868C0A7
:101200002B43164DDFF86490A84207D0B04205D0BA
:10121000B84203D0604501D0484506D123F0080804
:10122000CB6843EA080323F00403A84207D0B04286
:1012300005D0B84203D0604501D0484505D14D697D
:1012400022F4407215438A692A43426084614968E6
:1012500041630362BDE8F0838FFFFEFF00000140A1
:1012600000040140004001400044014000480140AA
:10127000F0B5026A22F010020262056A42688369D0
:10128000194C1B4E23400C6823F4407343EA04249A
:1012900025F020038D6843EA0513144DA84201D0C0
:1012A000B04206D1CF6823F0800343EA071323F04E
:1012B0004003A8420AD0B04208D00E4DA84205D043
:1012C0000D4DA84202D00D4DA84207D14D6922F420
:1012D000406242EA85028D6942EA85024260846189
:1012E000496881630362F0BDFF8FFFFE000001408B
:1012F000000401400040014000440140004801401A
:10130000F0B5026A22F480720262026A4368C4691C
:1013100022F40072184E24F073050C682C438D687B
:1013200042EA0522134DA84201D0B04206D1CF684F
:1013300022F4006242EA072222F48062A8420AD024
:10134000B04208D00D4DA84205D00D4DA84202D0A4
:101350000C4DA84207D14D6923F4405343EA0513CD
:101360008D6943EA05134360C4614968C163026241
:10137000F0BD0000000001400004014000400140B9
:10138000004401400048014030B5026A22F4805216
:101390000262036A4268C46923F400530D6824F4AE
:1013A000E64444EA05248D6843EA05330C4DA8421F
:1013B0000BD00C4DA84208D00B4DA84205D00B4DC8
:1013C000A84202D00A4DA84204D14D6922F48042BD
:1013D00042EA85124260C46149680164036230BD1B
:1013E0000000014000040140004001400044014071
:1013F0000048014030B5026A22F480320262046A79
:101400004268436D24F4003423F070050B682B43CD
:101410000D8944EA05440D4DA8420BD00C4DA8425D
:1014200008D00C4DA84205D00B4DA84202D00B4D60
:10143000A84204D14D6922F4803242EA052242607A
:10144000436549688165046230BD000000000140C9
:1014500000040140004001400044014000480140B8
:1014600030B5026A22F480120262046A4268436D57
:1014700024F400140D6823F4E04343EA05230D89A6
:1014800044EA05540C4DA8420BD00C4DA84208D09C
:101490000B4DA84205D00B4DA84202D00A4DA842E0
:1014A00004D14D6922F4003242EA8522426043654C
:1014B0004968C165046230BD00000140000401407C
:1014C00000400140004401400048014001490860DB
:1014D000704700004004004070B5046A24F0010425
:1014E00004628469056A154EB04214D0B0F1804F91
:1014F00011D0134EB0420ED0124EB0420BD0124E4D
:10150000B04208D0114EB04205D0114EB04202D0C8
:10151000104EB04203D124F00304144301E044F020
:1015200001041A0724F0F00425F00A0301F00A016F
:10153000194344EA12628261016270BD00000140F9
:101540000004004000080040000C0040000401407E
:10155000001800400040014030B5046A24F0100437
:1015600004628569046A25F4407545EA022222F482
:1015700070454FF6FF7202EA033224F0A003A02464
:101580002A43826104EA01111943016230BD90F8D7
:101590003410C90706D001684A68836B22F4003210
:1015A0001A434A6090F83410890706D501684A68E2
:1015B000C36B22F480321A434A6090F83410490712
:1015C00006D501684A68036C22F480221A434A60F7
:1015D00090F83410090706D501684A68436C22F474
:1015E00000421A434A6090F83410C90606D50168D3
:1015F0008A68836C22F480521A438A6090F834100F
:10160000890606D501688A68C36C22F400521A4321
:101610008A6090F83410490611D501684A68036D54
:1016200022F480121A434A60016DB1F5801F06D181
:1016300001684A68436D22F4C0021A434A6090F878
:101640003410090606D501684A68806D22F400222C
:1016500002434A607047F8B500250446C567FEF7A7
:1016600073FE0746206800686FF07E46000708D5C5
:1016700000223B464FF400112046009600F0FAFA93
:1016800060B92068006840070AD500223B464FF445
:1016900080012046009600F0EDFA08B10320F8BD65
:1016A000202084F8790084F87A00002084F87850AB
:1016B000F8BD10B5806B0021A0F86A10A0F8621088
:1016C000FFF718FB10BD01680A6822F490720A60E7
:1016D00001688A6822F001028A60202180F87A106D
:1016E000704710B5B0F86C2090F87A300168222B62
:1016F00005D0088B40F008000883022010BD898CBB
:101700008368B3F5805F01D103696BB11140426E0C
:10171000531C43661170B0F86A10491E0904090C85
:10172000A0F86A1007D015E0436E11401980416E91
:10173000891C4166EFE701680A6822F490720A602A
:1017400001688A6822F001028A60202180F87A10FC
:10175000FEF7FFFD002010BD2DE9F04F04460068A4
:101760008025FD4B0021D4F810C087B0A6680F4635
:10177000D4F81C8046EA0C06D4F814C0A26A4CEADD
:10178000080C46EA0C0632430668DFF8D0C306EAC6
:101790000C061643066020684268E66822F4405250
:1017A000324342602268A0699A4201D0266A3043DF
:1017B000A66AB6F1005F04D1D4E90B6C46EA0C06C8
:1017C00030439668DFF898C306EA0C060643966035
:1017D0002068C26A666A22F00F023243C262E14E9A
:1017E0002068E14AB04210D1126802F03802182A8B
:1017F00074D005DCCAB3082A7AD0102A47D179E020
:10180000202A7BD0282A7CD17AE0D84EB04209D158
:10181000126802F00702062A73D2DFE802F0536969
:101820006B6D6F71D24EB04209D1126802F007029F
:10183000062A66D2DFE802F0465C5E606264CD4E46
:10184000B04209D1126802F00702062A59D2DFE835
:1018500002F0394F51535557C74EB0420BD1126861
:1018600002F00702062A4CD200E00EE0DFE802F0A8
:101870002A4042444648C14EB04209D1126802F0A3
:101880003802182A38D0BBDCB4E74FF0010538E045
:10189000BB4EB04209D1126802F00702062A30D2CC
:1018A000DFE802F01026282A2C2EB64EB0420BD1CB
:1018B000126802F00702062A23D2DFE802F00319B9
:1018C0001B1D1F2100251CE098421AD1A64A121D9B
:1018D000126802F00702062A13D202E00CE007E0C9
:1018E0000CE0DFE802F0030507090B0D022508E014
:1018F000042506E0402504E0082502E0102500E06C
:101900002025DFF864B2A04E9842DFF880A2ABF148
:10191000540B73D1102D31D006DC022D09D0042DCB
:101920000AD0082D2FD111E0202D29D0402D2AD109
:1019300007E0FEF789FD13E06846FEF79BFD01987E
:101940000EE003A8FEF714FE049809E0DBF800108F
:101950005846890610D50068C0F3C1012AFA01F083
:10196000002811D06168894601EB410181420AD803
:10197000B0EB093F07D808E05046F3E78448F1E7A9
:101980004FF40040EEE7012733E1102D4FF000083F
:101990004ED006DC022D0FD0042D15D0082D04D119
:1019A0002DE0202D4AD0402D13D00127794AA0F5F3
:1019B0004071914270D9E6E7FEF746FD626A002366
:1019C000414636F812200DE06846FEF753FD0198B7
:1019D00003E003A8FEF7CCFD04980023616A36F803
:1019E00011201946FEF7BAFC62680902030241EAB7
:1019F00010615008181841EB080115E032E0DBF8DF
:101A000000105846890609D500680023C0F3C101BB
:101A10002AFA01F0616A36F8112015E0606A0023A5
:101A200036F8102050460FE00023FEF797FCBDE784
:101A3000606A002336F81020554805E0606A0023EC
:101A400036F810204FF400400021FEF787FC090211
:101A5000020241EA10614FEA590010184A4641EB70
:101A60000801E1E7E3694FF4004293424DD1082DAC
:101A700023D005DC8DB1012D12D0042D06D112E04A
:101A8000102D35D0202D3AD0402D11D0012721F036
:101A90000F00C1F3420108435AE0FEF764FC16E070
:101AA000FEF766FC13E06846FEF7E4FC01980EE0E2
:101AB00003A8FEF75DFD049809E0DBF80010584626
:101AC000890608D50068C0F3C1012AFA01F0616AED
:101AD00036F8111010E0606A36F81010BAFBF1F019
:101AE0004100606801EB5001B1FBF0F081B2CEE73C
:101AF000606A36F810102648B0FBF1F0F0E7606A33
:101B000036F81000B2FBF0F0EAE7082D4AD00ADC04
:101B10000DB3012D43D0042D7FF44DAF6846FEF781
:101B2000A9FC019809E0102D52D0202D55D0402D50
:101B3000F2D103A8FEF71CFD0498616A36F8111073
:101B4000B0FBF1F1606801EB5001B1FBF0F080B245
:101B50002168C8604DE01FE0000C0058F369FFCF1A
:101B6000FFF4FF11001001405444025800440040AB
:101B700000480040004C004000500040001401406C
:101B800000780040007C0040D81C00900090D003FA
:101B900000093D00FFFC0F00FEF7E5FBCDE7FEF777
:101BA000E7FBCAE7DBF80020594692060AD5096828
:101BB000C1F3C1022AFA02F1626A36F81220B1FBBF
:101BC000F2F20FE0616A36F81120BAFBF2F209E096
:101BD000616A36F811200949F1E7616A36F8111097
:101BE000B2FBF1F2616802EB5102B2FBF1F189B292
:101BF000C16007B03846BDE8F08F000000093D0025
:101C000090F87910212901D002207047B0F86210B5
:101C100021B18168B1F5805F13D014E001680A68D2
:101C2000920004D58A6822F400028A6003E00A6800
:101C300022F080020A600068016841F04001016002
:101C40000CE0016961B1C16D4A1CC2650268097886
:101C50001185B0F86210491EA0F86210002070478C
:101C6000C16D02680988C1F308011185C16D891C25
:101C7000C165EEE72DE9F0411E4617468846044649
:101C8000069D1CE0681C1AD025B1FEF75DFB801B89
:101C9000A84214D92068016821F4D071016020683D
:101CA000816821F001018160202084F8790084F8A6
:101CB0007A00002084F878000320BDE8F0812068D5
:101CC000C16938EA010004D00020B842DAD000200F
:101CD000F3E70120F9E7FEE7010002000400060037
:101CE00008000A000C0010002000400080000001E5
:040000050800029954
:00000001FF
